:020000040000FA
:020000000C28CA
:08000800A0000308A10021087B
:100010008300A00E200E0900703083169000FF3080
:1000200081008312830185010730990083169F01A7
:100030000E3085008312AE010516DF204E20CC3035
:1000400066204430662063004E20CC306620BE30EF
:10005000662081202908AB0081202908AC004E20B1
:1000600005128516DF200A30AD00A020AA30AB2093
:100070000130AB202C08AB202B08AB20AD0B352872
:10008000851285016300AE0A64302E02031D4228EA
:100090001B2800000000A30B492800348316051517
:1000A0008312A9018312051183160511831263308F
:1000B000A30049208316051583121330A30049209D
:1000C000051DA90A4F30A30049200034A9000830BB
:1000D000AA00831205118316051183120000000087
:1000E000000000000000A90C031805150B30A30048
:1000F000492083160515831200000000AA0B692809
:100100000034A9010830AA008312051183160511D5
:1001100083120000000000000000000000008316B1
:1001200005158312000000000000000005080439D6
:10013000FF3EA90C0930A3004920AA0B84280034F3
:100140000830A700CD20CD20CD20A70BA228051474
:10015000CD2005100800A6000830A700CD20A60D70
:10016000031C0514CD200514CD200510A70BAE28C7
:1001700008000530A500A401A301A30BBD28A40B12
:10018000BC28A50BBB2808000530A4004130A30003
:10019000A30BC828A40BC62808002D30A4000130EA
:1001A000A300A30BD128A40BCF2808000130A40082
:1001B0001130A300A30BDA28A40BD8280800A03024
:1001C000A400CF30A300A30BE328A40BE128080070
:02400E008C3FE5
:00000001FF
